:020000020000FC
:0200000073C0CB
:0200160018953B
:10001A0015C00F931F932F933F930FB7B49908C03E
:10002A0020916000203009F003C011E010936000B5
:10003A000FBF3F912F911F910F9118954F935F9387
:10004A000F931F935FB74091670045300CF403C0CC
:10005A00442740936700403081F493989498959888
:10006A000EF002C00BE002C000916500002311F0FF
:10007A00929A01C09298B0D12BD1413081F49298D2
:10008A00949895980091640030916500032B11F0C3
:10009A00939A01C09398009164009ED119D142307D
:1000AA0059F4929893989598949A0091630094D1F0
:1000BA00002D0F77002E0CD1433041F4929893987B
:1000CA009498959A00916B0087D102D143954093F9
:1000DA0067005FBF1F910F915F914F9118950FEDC8
:1000EA000DBF0FE701BB01EE07BB0CE108BB02E045
:1000FA0000BF05E003BF09E106BF00E20BBF0CE148
:10010A0000BD11241092670000E00093600000E037
:10011A0000936C0005E000936D000FE000936E0001
:10012A0001E000936F0000270093690000936A00C2
:10013A0000EF00936B006ED000917000083209F452
:10014A0005C012E01093600056D101C050D180E082
:10015A0090E000916000003031F4969823D147D0A6
:10016A0001E009BF1CD0013019F496981BD1BCD00C
:10017A00023079F7969AEDCFEE24FF1841E1001F7D
:10018A00111F4A9509F40895EE1CFF1CE21AF30A9E
:10019A0020F4E20EF31E8894F2CF0894F0CF0F9366
:1001AA001F932F933F934F935F936F93009169002F
:1001BA0010916A0020916B003CE140E250916F007F
:1001CA000EF001C00195552309F409C030170CF44B
:1001DA0002C0909A04C004170CF401C090986F9161
:1001EA005F914F913F912F911F910F9108951F9306
:1001FA0065D05CE034E34DEF19D15CE034E34DEFB8
:10020A0015D112D010916900812F10916A00912F97
:10021A001F9108950F9376D003E3802E88D0A0E72C
:10022A00B0E0A6D00F9108950F931F932F933F9399
:10023A004F9368D00CEC802E7AD00EEB802E77D0BC
:10024A00A9E6B0E095D0AAE6B0E092D01091690094
:10025A0020916A002F93287F283F11F0E89409C063
:10026A002F9168941095209531E0130F30E0231FE9
:10027A0001C02F91269517952695179526951795BE
:10028A0026951795309169000EF43195432F3F70EA
:10029A00432F330F330F330F440F340F36953695F0
:1002AA00369536951093690020936A0030936B0057
:1002BA004F913F912F911F910F9108950F9322D043
:1002CA000CEC802E34D004E4802E31D00F910895A6
:1002DA000F930FB800E40EB90BE10DB9769BFDCF71
:1002EA00C09AC0980F9108950F938CD0B29B019633
:1002FA00B39B0197B49B01C003C000E00093600068
:10030A000F910895F894B99A33E04EEB8BD0B998CF
:10031A0030E04AE887D005D033E042E383D07894CE
:10032A000895B19B716002C0B1997E7F08950F93C1
:10033A001F93082D18E0069508F458F0F894B99A16
:10034A0030E046E76FD0B99830E042E16BD078945C
:10035A000AC0F894B99A30E04AE064D0B99830E01B
:10036A004EE760D078941A9531F71F910F9108954E
:10037A000F931F93002718E0F8940695B99A30E076
:10038A004AE050D0B99830E040E14CD0B1990068C9
:10039A0030E04CE647D01A9581F70C9378941F9178
:1003AA000F910895F8945F9354E0A3E6B0E0809328
:1003BA0061009093620000916100109162002AE04E
:1003CA0030E0DADEED9200936100109362005A95F4
:1003DA0091F75F91789408950F931F93E0E6F4E004
:1003EA001127E00FF11F04901F910F910895C59AEC
:1003FA0022D0C5980895C59A1ED01DD01CD01BD0F6
:10040A00C59808950F931F932F932AE01FEF0FEFBC
:10041A000A95F1F71A95D9F72A95C1F72F911F91E5
:10042A000F91089541503040E8F708954150304007
:10043A005040E0F708950F931F932F9326E00FEF94
:10044A001FEF1A95F1F70A95D9F72A95C1F72F9157
:10045A001F910F910895C0F9A4B0999282F88090E3
:02046A009CBF35
:00000001FF
